:030000000201B644
:03000B000206CF1B
:0300400001FF10AD
:020043000201B8
:0300330002018047
:100100000206DF00020779000207790002072600D5
:1001100002074F0002077900020779000207790001
:1001200002077900020779000207790002077900C7
:1001300002077900020779000207710002077900BF
:1001400002077900020779000207790002077900A7
:100150000207790002077900020779000207790097
:100160000207790002077900020779000207790087
:100170000207790002077900020779000207790077
:1001800053D8EF3290E6A3E020E22A90E690E0B464
:10019000002390E691E0B41F1C759AF0759B0075E2
:1001A0009D0A759E87781FE59CF59FD8FAD2077443
:1001B0008090E691F02275816F1210DF1202793083
:1001C0000C1FE4120BD24016D20B120BC090E61A91
:1001D000740C200D027404F0120A861208F5120342
:1001E000B63006031203E130040843870100000023
:1001F000C20430080512083D80E731843007091237
:10020000087930070312077AE55754046554606291
:100210006554F554E5567050D55557755510200B5B
:100220001CE4120BD2404BD20B120BC090E61A7496
:100230000C200D027404F0120A86020272E53312D9
:100240000BC26006120BCE020272C20B300C16906B
:100250000AB07401F0A3E4F0900AC674FFF0A3F0B2
:10026000A3F01203B6020272D55607E4120D7E12F5
:100270000BCE000000000021E1C206C204C205C28C
:1002800000C201C20CC20D753400D20E900040E0D5
:10029000600FD20CA3E0F9A3E0C9900AB0F0A3E983
:1002A000F0755600755400755510C20B120BC074D2
:1002B000FF90E65DF090E65FF0754055754153752F
:0802C0004242754353E4F5537B
:1002C800F550F551F552F537F54FF55990E680E0C0
:1002D80020E70C900AB3E4F0744078000202F19031
:1002E8000AB37401F074007802900ACEF0C8A3F043
:1002F800C8900AD5F0C8A3F0C890E625F0C8000059
:100308000090E624F0C8F5358836C207C208D2E85E
:1003180043D820538EF85391EF90E600E054FDF057
:1003280090E6687408F090E65CE04409F00000008C
:1003380090E61274A0F090E61474E0F0E490E610F1
:10034800F090E611F090E613F090E615F090E618BC
:100358007400F000000090E619F000000090E61B21
:10036800F000000090E61A740C200D027404F000EE
:10037800000090E6917480F000000090E69174808F
:10038800F000000090E6917480F000000090E69183
:100398007480F000000090E65E7440F0D2AF90E602
:1003A80080E04402F0758901758810D2A92290E690
:1003B80080E04408F0F0E04402F07FDC7E0512069D
:1003C800B990E680E054F7F07E187FFF1206AB2064
:1003D8000606DFF8DEF680D62290E6B9E0700B90CC
:1003E800E6B8E024DF700002042C147003020498BD
:1003F80024FE70030204F324FB70030205651470E5
:10040800030205761470030205921470030205A115
:100418002405700302063790E6B8E030E6030205CB
:0D042800B602067B90E6B8E0247F60231446
:1004350060302402705AA205E43325E0FFA200E4EF
:10044500334F90E740F0E4A3F090E68B7402F0029E
:100455000682E490E740F0A3F090E68B7402F00288
:10046500068290E6BCE0F45480C4FFE05407200106
:1004750002701D2F25E024B4F58275837FE054FEBC
:1004850090E740F0E4A3F090E68B7402F002068258
:1004950002067B90E6B8E024FE6007240260400275
:1004A500067B90E6BAE0704390E6BCE0F45480C465
:1004B500FFE0540720010270322F25E024B4F582B5
:1004C50075837FE4F090E6BCE05480131313541F4A
:1004D500FFE054072F90E683F0D2E5F00206829004
:1004E500E6BAE0B40105C20502068202067B90E683
:1004F500B824FE60072402605802068290E6BAE03E
:10050500705B90E6BCE0F45480C4FFE05407200122
:100515000270D82F25E024B4F58275837F7401F02D
:10052500C083C08290E6BCE05480131313541FFFB0
:10053500E054072F90E683F0D2E5F0D082D083EF28
:1005450020E407A37401F0020682E0D2E1F002067E
:100555008290E6BAE0B40105D20502068202067B66
:1005650090E740E4A20133F090E68B7401F00206B7
:0A0575008290E6BAE0600BB40110BA
:10057F00D20112068C020682C20112068C0206827A
:10058F0002067B90E740E530F0740190E68BF002B5
:10059F0006822001030205B390E6BAE0F530120699
:1005AF008C02068202067B90E6B9E0B41028E43094
:1005BF000B0E90E6BCE0F9C3E53399E44002E53455
:1005CF0090E740F0A3E533F090E68AE4F090E68BF5
:1005DF007402F0020682B4114990E6BCE0B53335DF
:1005EF00E5567015E533120BC2602A7403120D7EA7
:1005FF00755604120D91120927120DAEE4900B3EA1
:10060F007D40C0E0120E8AEFF0A3EEF0A3D0E0041D
:10061F00DDF0120DB590E6B3740BF0A3743EF0024B
:10062F000682B4120002068290E6BBE024FE60143C
:10063F0014601E2402703590E6B3740AF0A374A6FA
:10064F00F002068290E6B3740AF0A374B8F00206C3
:10065F008290E6BAE023F9900AD893C90493C9901F
:10066F00E6B3F0A3E9F002068202068290E6A0E06C
:10067F004401F090E6A0E04480F0C2062290E683A9
:10068F00E47F08F0D2E5F0C2E505E0DFF67F0874FD
:10069F0010F0D2E5F0C2E505E0DFF6227586009096
:1006AF00FB50A3E582458370F9228E318F32E532FC
:1006BF001532AE31700215314E6004D1AB80EF228E
:1006CF000557C0E0E5586005147000F558D0E032CA
:0406DF00C0E0C08334
:1006E300C082C085C084C086C0D074EF529190E6AA
:1006F3005D7401F090E6B8E0B42117A3E0B4FF12F3
:10070300120A541210D975816F51B9D1821207257B
:1007130021E1D206D0D0D086D084D085D082D083B8
:10072300D0E032C0E0C083C082C085C084C086D21E
:10073300045391EF90E65D7408F00000000000D0D0
:1007430086D084D085D082D083D0E032C0E0C0830D
:10075300C082C085C084C0865391EF90E65D74105B
:10076300F0D086D084D085D082D083D0E03253912C
:10077300EFF5A105593232754D00754E00754F00E6
:10078300300B0BE5567019E533120BC2700574017B
:100793000207AC7403120D7E120D913184120927E6
:1007A3007556041210D612093DF54C300A42200941
:1007B30003120863300D1B90E6AFE0F990E6B0E05A
:1007C300F849600BE5AA20E6FB90E6487406F002C0
:1007D3000835E54D454E605AC333F9E43390E69846
:1007E300F090E699E9F090E6A5E030E2F9020835E9
:1007F30020093FAD48AC49754800754900E4C54F31
:10080300C333F9740033F8496006748090E691F0BD
:10081300EDC399FDEC98FC40194D601690E6A3E0FA
:1008230020E2F990E690E0F890E691E0F97480F028
:1008330080DED208C20712083D2290E6A5E05409E3
:07084300701DC20890F800CF
:10084A0079407F0DE7F009A3DFFA90E698E4F0908B
:10085A00E699740DF01210D922AC48E549C313CCBD
:10086A0013FD74003400F548120F2C7549002275E7
:10087A009A0A759B8790E67BE0B45528E0B4532426
:10088A00E0B44220E0B4431C79447F04E0F709DF76
:10089A00FB7F04D209E0F76002C20909DFF7E0A290
:1008AA00E7920A22C20790E6A5E04401F090E6A387
:1008BA00E04401F022E5AC30E1FB90E6047480F0FC
:1008CA000000007402F00000007400F000000074E0
:1008DA008090E691F000000090E691F00000009010
:1008EA00E691F000000090E691F022E533120BC287
:1008FA00602A120DAE7437900B2E7D04C0E0120EE2
:10090A008AEF70027430F0A3A3EE70027430F0A381
:10091A00A3D0E004DDE6120DB5120BCE22740679DF
:10092A00A0120CB974017900120CB9740E7908126C
:10093A000CB9221201847407120CB254886009E5BA
:10094A0056740170EE740122740479FF120CB974A2
:10095A000579FF120CB9740779A0120CB912018437
:10096A007407120CB254806009E556740170EE7473
:10097A0001221201847407120CB254087009E55658
:10098A00740170EE740122900A967E067F00120DA1
:10099A0051120184120D6C701A740E120CB25408A2
:1009AA007007E55670EB7401227402120CB21460DF
:1009BA00C180DE7407120CB27402120CB2540370B6
:0A09CA0008120A1A12100180C81466
:1009D40070057402020A1914702F30092474041269
:1009E4000CB2FC7405120CB2C313CC13FD7F0012BD
:1009F4000CD8DDF9EC60A01C80F3809B7402020A21
:100A040019120A1A120F2C808E7407120CB2540198
:100A14006003000000227404120CB2FC7405120C72
:100A2400B2FDD20975F0007948E7C39C42F0F7099A
:100A3400E79D42F0F709E7940042F0F709E79400D4
:100A440042F0F7E5F06002C209EDC313CC13FD22B6
:100A5400300B2EE556602A7407120CB224B06021C4
:100A6400740E790C120CB91206AB740E7908120CC0
:100A7400B9780079007407120CB230E704D9F6D8BB
:030A8400F4222237
:100AA6001201000200000040C90A00000000010215
:100AB600030109022000010100C0320904000002FE
:100AC600080650000705860240000007050202409E
:100AD60000000AE00AE40B040B2C040309042003BB
:100AE6004D006900630072006F00200053006F0024
:100AF6006C007500740069006F006E0073002803B7
:100B06004200410043004B005000410043004B00AF
:100B160020005500530042003200200043006100CF
:100B260062006C00650012033000300030003000B7
:080B36003000300030003000F7
:100BC000E422F533120BF074004002740122120C7F
:100BD0004322F533120C43120BF050080533E53372
:100BE00070F5D322120CD0F534120BCEE533C322AC
:100BF000E533F4F59075B0F0120C3EF4F590120C5C
:100C00003EB2B7120C3EB2B7120C3EB2B7120C3E57
:100C1000C2B5E533540765B054077020D2B5E5334B
:100C2000F4540765B054077013D2B7C0017910743B
:100C300004120CC8D001C3E533020C3DD322C0011D
:100C4000D00122C2B7120C3E75B00022C2B4F5909A
:100C5000120C3EB2B522C2B4F590B2B622D2B4752F
:100C6000B300B2B6120C3EE590C2B475B3FF22D207
:100C7000B4E583F59AE582F59B75B300B2B61F1211
:100C80000C3EE590F59CB2B6DFF5120C3EE590F512
:100C90009CC2B475B3FF058622C2B4E583F59AE51C
:100CA00082F59B120C3EE59CF59000B2B6DFF40590
:100CB00086224440120C4C80A44440120C4CE98023
:100CC000954400120C4C80954400120C4CE980862F
:100CD000740B120CC1543F2279507404120CC8EFEB
:100CE0004440120C4C120C5DCF4440120C4C120CC0
:100CF0005DFE79107404120CC82279507404120C31
:100D0000C8EF4440120C4CED120C56EF4440120C4C
:100D10004CEE120C5679107404120CC822EE23FE0D
:0B0D2000E534B405127438120C4CEEE0
:100D2B00120C567400120C5674104FFF7950740449
:100D3B00120CC8EF4440120C4CEEFF120C6F7910E2
:100D4B007404120CC82279507404120CC8EF44407E
:100D5B00120C4CEE23FF120C9979107404120CC870
:100D6B0022740B120CC15480227405120CC154C096
:100D7B0023232254030303F97405120CC1543F4976
:100D8B00F97405020CC87405120CC14408F97405FA
:100D9B00020CC87406020CC1C0E0F97406120CC830
:100DAB00D0E022120D9E440880EE120D9E54F78067
:100DBB00E7120D9E440480E0120D9E54FB80D91265
:100DCB000DBC120DF960FB80EFC0E0C0F054016068
:100DDB00027402F5F0120D9E54FC45F0120DA34463
:100DEB0001120DA354FE120DA3D0F0D0E02274001B
:100DFB00120CC154806002740122120DBC740112DA
:100E0B000DD414120DD4120DD404120DD4120DD412
:100E1B00120DD4120DD4120DD4120DD4120DC322F7
:100E2B00120DBC7401120DD414120DD4120DD41268
:100E3B000DD4120DD4120DD4120DD4120DD4120DDB
:100E4B00D4120DC322C0E0120DBC7401120DD47468
:100E5B0000120DD47401120DD4D0E02323237B0692
:100E6B00120DD423DBFAEE7B0823120DD4DBFAEF41
:100E7B007B0823120DD4DBFA120DC3120DCA22C04C
:100E8B00E0120DBC7401120DD4120DD414120DD43A
:0D0E9B00D0E02323237B06120DD423DBFAC5
:100EA8007B08C0E07400120DD4120DF913D0E033A2
:100EB800DBF0FE7B08C0E07400120DD4120DF913AC
:100EC800D0E033DBF0FF120DC322120DBC74011207
:100ED8000DD414120DD4120DD404120DD414120D05
:100EE800D4120DD4120DD4120DD4120DD4120DC378
:100EF800120DCA120DBC7401120DD414120DD412A5
:100F08000DD4120DD404120DD4120DD4120DD41216
:100F18000DD4120DD47B1014120DD4DBFB120DC3AB
:100F2800120DCA22E534B405137438120C4CEDC303
:100F380033FEEC33CE120C56EE120C567950740474
:100F4800120CC87440A934B905024410120C4CD2D2
:100F5800B475B300ED4C700DC2B475B3FF7910745D
:100F680004120CC822E54D254DF8E54E354EC8242F
:100F780000F59BE834F8F59AE536C313F8E5351320
:100F8800C3954DF9FBE8954EF8FAEDC399EC9840F6
:100F980009754D00754E00020FAEEDFB254DF54D60
:100FA800ECFA354EF54EEDC39BFDEC9AFCB2B690CB
:100FB800E6A5E020E3FCEBC39401FBEA9400FA4BBE
:100FC8006017E590B2B6F59C00E590B2B6F59C00C6
:100FD80000DBEFEA60031A80E9E590B2B6F59C0001
:100FE800E590F59CE54D454E700C90E698E536F099
:030FF80090E699E7
:100FFB00E535F0020F5C79507404120CC874401282
:10100B000C4CC2B4E54F6029FAE59FF590B2B6E5FA
:10101B009FF590B2B6DAF2748090E691F074F0F529
:10102B009D7400F59EEDC3954FFDEC9400FC754F40
:10103B000074F0F59D7400F59E7B00EC604B7A40DC
:10104B0090E6A3E020E2FCE59FF590B2B6E59FF5B4
:10105B0090B2B6E59FF590B2B6E59FF590B2B6E5C6
:10106B009FF590B2B6E59FF590B2B6E59FF590B2BD
:10107B00B6E59FF590B2B6DACE748090E691F07437
:10108B00F0F59D7400F59EDCB5ED603790E6A3E0BE
:10109B0020E2FC90E690E0C313FA90E691E013C3D4
:1010AB009DF54FE59FF590B2B6E59FF590B2B6DD95
:1010BB00F2E54F700E748090E691F074F0F59D742C
:0B10CB0000F59E79107404120CC8227E
:1010D600D28522C28522B2852290E6007410F09055
:1010E600E60174C0F090E6C3743FF090E6C2743F28
:1010F600F090E6F37440F075B3FF75B5F075B2EF96
:101106001210D975B4FF75B6FF12119B2290E60135
:1011160074F2F075B54090E6C2743FF090E6C37481
:1011260038F090E6C17400F090E6C074E4F090E602
:10113600F5F02290E60174C0F090E6C3743FF0909B
:10114600E6C2743FF075B5F02204010157001101A3
:101156005300010053003F035300040103570011DD
:10116600035300130357003F0757000401015700BC
:1011760011015300010257001F01570006010357D2
:10118600001303573F220353002303560027035738
:10119600003F03570090E60174C2F07592E4787F31
:1011A6007980E4F218D9FC75921A78007980E4F215
:1011B60008D9FC90114F75921A78007904E0A36063
:1011C60013FA7B04E0A3F2E82408F8DBF7E8C394FB
:1011D6001FF8DAEEE8242054E0F8D9E1787F797F29
:1011E6007A8075921AE360047592E4F21819DAF2BD
:1011F600787F797F7A8075921AE3FB7592E4E2C371
:101206009B6004EBF280E91819DAEB90E6F5F090B2
:09121600E60174C0F0759200229B
:00000001FF
